:020000040000FA
:06000000653002303A28D1
:08000800A000030EA100831209
:100010008B1C32288B1031181428B11C3228643004
:10002000010203183128182800001628172818285C
:1000300019281A281B281C281D281E281F283110A3
:10004000B114A810031005190314AA0DA90DA80DC9
:10005000B00B322831152A08AF002908AE00280855
:10006000AD00B11081010B11210E8300A00E200EF6
:02007000090085
:0C007400203084008001840A6030040207
:10008000031C3C281230B0009F218316FF239000F0
:10009000831283160C308505870183128501870141
:1000A000073099000030831691009F008312C830FA
:1000B00083168100831231309000003083168C004B
:1000C000831210308B002F2281018E018F010B11C2
:1000D0008B100B108C018B177B2031199120B30BE7
:1000E0007928031085190314B90DF030390203196A
:1000F000162130226C286400311808000B1D0800FE
:100100000B11B11031141230B000051D8C283214BF
:10011000831601138312080032108316011783120D
:10012000080031110130B70085148B1320303707D8
:1001300083169B001C141A088312A400A500C0306B
:10014000A5061030370783169B001C141A0883126B
:10015000A3000030370783169B001C141A08831273
:10016000A2008B17321CBA2822090339A200A30966
:10017000A409A50922082D02031D102923082E0217
:10018000031D102924082F02031DE2280130370225
:10019000031DCD283D143E14B42102303702031D47
:1001A000D428BD143E14BC2103303702031DDB28C4
:1001B0003D153E14C42104303702031DE228BD154D
:1001C0003E14CC2125082F02031D032901303702DC
:1001D000031DED283D103E14D42102303702031DCB
:1001E000F428BD103E14DC2103303702031DFB2828
:1001F0003D113E14E42104303702031D0229BD11D4
:100200003E14EC2110295F08AB3C03191029321869
:100210000C292F1810290F292F1C10290F29F42120
:10022000B70A053037020318080095280130B600D8
:10023000B300B400B500B70085018701B1131922DE
:100240007B20B30B5129031085190314B90DF0302D
:10025000390203197829B41F8501B41F8701B41F1F
:100260008510B40B5129B50B51290230B50001306E
:1002700037020319FD21023037020319022203302D
:10028000370203190B2204303702031914223708EE
:10029000B6080319B60003194F298514B603FA30BE
:1002A000B400311D20293111321C5B292D0903397D
:1002B000AD00AE09AF092F1CB1132F1C2029B11BB3
:1002C00020292E182029B1178B1320303707BB00A7
:1002D0002F08BA008C2110303707BB002E08BA0057
:1002E0008C2100303707BB002D08BA008C218B17FA
:1002F0001D2285018701B70AB60105303702031CAC
:1003000020292F2208003E1C08003E101030BB00A0
:100310003D08BA008C2108008B133A0883161C157F
:100320009A003B089B0055309D00AA309D009C140C
:1003300064009C1898291C1183128B1708008316DF
:1003400000309B001C141A088312DF008316203033
:100350009B001C141A088312C1000130C11BC1008C
:10036000C1080319C1000800071287164008410799
:10037000D0000F08D100080005128715400841077A
:10038000D2000F08D3000800071185164008410766
:10039000D4000F08D5000800071087144008410753
:1003A000D6000F08D700080087120716400841073B
:1003B000D0000F08D100080087110516400841073A
:1003C000D2000F08D3000800851207154008410726
:1003D000D4000F08D5000800871007144008410713
:1003E000D6000F08D70008000712051207110710E2
:1003F000871287118512871008003F09303987005E
:10040000BF000800380910398500B8003F090839D5
:100410008700BF000800380920398500B8003F096F
:1004200004398700BF0008003F0903398700BF0077
:100430000800B801BF01BF160800B801BF010130B4
:100440003702031D242ABF1502303702031D292A53
:10045000B81603303702031D2E2ABF140800080007
:1004600050084002031D3A2A51080F02031C3A2A81
:100470000712871252084002031D442A53080F0234
:10048000031C442A0512871154084002031D4E2AFA
:1004900055080F02031C4E2A071185125608400208
:1004A000031D582A57080F02031C582A07108710EB
:1004B0000C1C08000C10C00A851008000C1C6C28CD
:1004C0000C10C00B6C284108C00085018701080092
:084000000100030005000100AE
:02400E00CC01E3
:10420000010003000300030003000200020002009B
:1042100002000000000000000000FF00FF00FF009F
:10422000000000000000000000000000000000008E
:104230000000C000C000C000C000FF00FF00FF0081
:104240000100C300F300CF00FF00C300F300CF0064
:10425000FF00C300F300CF00FF00FF00FF00FF00DE
:10426000FF00FF00FF00FF00FF00FF00FF00FF0056
:10427000FF00FF00FF00FF00FF00FF00FF00FF0046
:10428000FF00FF00FF00FF00FF00FF00FF00FF0036
:10429000FF00FF00FF00FF00FF00FF00FF00FF0026
:1042A000FF00FF00FF00FF00FF00FF00FF00FF0016
:1042B000FF00FF00FF00FF00FF00FF00FF00FF0006
:1042C000FF00FF00FF00FF00FF00FF00FF00FF00F6
:1042D000FF00FF00FF00FF00FF00FF00FF00FF00E6
:1042E000FF00FF00FF00FF00FF00FF00FF00FF00D6
:1042F000FF00FF00FF00FF00FF00FF00FF00AA001B
:00000001FF
